:1000000002C0189518958FE181BD87E181BD8FED04
:100010008DBFC0ECE8EB4E2EDD275D2EEEE7F0E065
:10002000A0E6B0E088278D933197E9F76624BC9A63
:10003000B898B998BA98C49883E090E0A0E68D93F8
:100040009C938DEF9FEFA2E68D939C9380E090E0D0
:10005000A4E68D939C9380E892E0A6E68D939C9312
:100060008EEA91E0AAE68D939C9382E593E0A8E660
:100070008D939C93E1E0F0E0ECD00027A6E38C9117
:1000800080FB0EF401E040E0041709F094C0002763
:10009000A6E38C9181FB0EF401E040E0041709F027
:1000A0002DC0A6E68D919C91A4E68D939C93A2E62B
:1000B00011961C90AAE64D915C91A4E60D911C91BD
:1000C0000417150717FC03C024F019F017C00CF42F
:1000D00015C084E0A4E6ED91FC91A8E3E2D084E1B0
:1000E00090E0C6D0A4E60D911C91A2E64D915C91E2
:1000F000040F151FA4E60D931C93D9CF0027A6E388
:100100008C9182FB0EF401E040E0041709F02DC051
:10011000A6E68D919C91A4E68D939C93A0E6119602
:100120001C90A8E64D915C91A4E60D911C910417DA
:10013000150717FC03C024F019F017C00CF415C004
:1001400084E0A4E6ED91FC91A8E3ABD084E190E0DB
:100150008FD0A4E60D911C91A0E64D915C91040F07
:10016000151FA4E60D931C93D9CF0027A6E38C910D
:1001700081FB0EF401E041E0041781E009F080E02A
:100180008F930027A6E38C9182FB0EF401E041E0FF
:10019000041781E009F080E09F918923882309F406
:1001A00009C084E0A6E6ED91FC91A8E37AD084E151
:1001B00090E05ED04BC00027A6E38C9181FB0EF44B
:1001C00001E040E0041709F009C084E0AAE6ED91DF
:1001D000FC91A8E366D084E190E04AD00027A6E332
:1001E0008C9182FB0EF401E040E0041709F009C095
:1001F00084E0A8E6ED91FC91A8E353D084E190E07F
:1002000037D00027A6E38C9181FB0EF401E041E09A
:10021000041781E009F080E08F930027A6E38C911A
:1002200082FB0EF401E041E0041781E009F080E078
:100230009F918923882309F409C084E0A6E6ED9103
:10024000FC91A8E32ED084E190E012D016CFF89470
:10025000FFCF88EE93E00CD03197D9F7089531970E
:10026000F1F70895689462F80895E89462F80895A3
:10027000EF93FF93EE27E82BE92B31F0EAEFF0E064
:100280003197F1F70197D1F7FF91EF91089591E040
:10029000882321F08894991F8A95E9F7892F9095F2
:1002A0000895BB27F4DF9C9198279C933197F1F731
:0602B00098279C930895BD
:00000001FF
